:1000000037C051C0CBC14FC04EC04DC04CC04BC01B
:100010004AC049C048C047C046C045C044C00902A4
:100020001200010100801909040000000000000016
:1000300012011001FF000008C016DC0504010102D6
:1000400000010E0355005300420061007300700070
:100050001C037700770077002E00660069007300AC
:10006000630068006C002E0064006500040309044E
:1000700011241FBECFE5D2E0DEBFCDBF10E0A0E669
:10008000B0E0EAEDF5E102C005900D92A436B107AB
:10009000D9F720E0A4E6B0E001C01D92A33CB2076E
:1000A000E1F76BD998CAACCFCF93DF9360918B0007
:1000B000635067FD14C0209188008CE090E0821BA3
:1000C0009109EC01C157DF4F809187008D3209F40F
:1000D00067C08091650087FDA9C010928B00809158
:1000E000610084FF3EC0609160006F3FD1F16930D4
:1000F00008F47EC068506093600090917B0088E8AF
:10010000892780937B0068E08091650087FD1CC093
:100110002091890030918A0086FF7FC0ACE7B0E073
:10012000F901962F84918D9331969150D9F78FEFE5
:10013000860F90E00196280F391F30938A00209394
:100140008900C4E0C60F5FC08CE790E06ED7682FCF
:10015000893008F4B1C08FEF80936000CEE1C09386
:10016000610094E186B3887181F49150D9F71092BF
:100170008C001092860080916400813019F0C1E0FB
:10018000C0936400DF91CF910895C1E09111C0E068
:1001900080916400C817B1F3F89499D87894F0CF9F
:1001A000683009F09ACF83EC80937B008AE58093D6
:1001B0006100109265008881807609F041C08A81D3
:1001C000109284009981911146C01092850024E814
:1001D00030E082E030938A00209389009F81911162
:1001E00004C09E81981708F4892F8093600075CF12
:1001F0001092600090917B0088E8892780937B00B3
:10020000611182CFC4E08CE790E0B1D0CC3009F42A
:10021000A6CF8FEF80936000A2CFD901ECE7F0E08A
:10022000962F8D9181939150E1F781CFCE017DD7AB
:100230008F3F01F1882309F450CF109260004DCF19
:10024000CE0194D48F3F51F6988197FD1DC090E860
:1002500090936500CACF953089F0963009F19830B7
:10026000D9F0993099F081E09A3009F080E024E8E3
:1002700030E0B0CF8EE1809361002FCF80938C006F
:1002800024E830E080E0A6CF8E81E1CF80938E001D
:1002900024E830E080E09ECF2EE830E081E09ACF85
:1002A0009B819130F1F09230A1F0933041F080E0E9
:1002B00090E49093650092CFC4E0C80FA4CF811161
:1002C00018C08CE690E090938A008093890084E0C7
:1002D000EFCF8EE190E090938A008093890082E1D5
:1002E000E7CF80E390E090938A008093890082E1D9
:1002F000DFCF813051F08230D1F682E490E09093EC
:100300008A00809389008EE0D3CF80E590E09093BF
:100310008A00809389008CE1CBCFAC9A8BB7806246
:100320008BBF0895A82FB92F8FEF9FEF1BC02D9182
:100330008227282F22952827722F26952695272752
:10034000239526952170782F892F82272195207C4F
:10035000922F22277695279597278227769527959E
:1003600097278227615018F7809590950895DADFD6
:100370008D939D930895A6E088279927AA9569F003
:100380000197E1F3B399FCCFB39BFECF81E09927AE
:10039000A6B3019611F0A871D9F70895CF93CFB7FE
:1003A000CF93C395B39BE9F7B39B0BC0B39B09C035
:1003B000B39B07C0B39B05C0B39B03C0B39B01C0F5
:1003C000D3C00F92DF93C0918800DD27C157DF4F64
:1003D000012EB39B03C0DF910F90E6CF2F930F93B5
:1003E0001F934F932FEF4F6F06B303FB20F95F93DB
:1003F0003F9350E03BE065C016B30126502953FD02
:10040000C89556B3012703FB25F92F7306B3B1F046
:100410005027102713FB26F906B22230F0F000C057
:1004200016B3012703FB27F90126502906B2243011
:10043000E8F54F77206816B30000F6CF50274F7DC0
:10044000206206B2102F000000C006B3002650291B
:10045000102713FB26F906B2E2CF4F7B06B32064C8
:1004600000C0DACF01265029187106B269F14E7F1B
:100470002160012F16B328C0002650294D7F06B2F7
:100480002260102F29C0012650294B7F06B224601C
:10049000012F2DC016B301265029477F2860000088
:1004A00006B22EC04F7E06B3206130C0422706B38D
:1004B000499300265029102706B24FEF13FB20F96D
:1004C000297F16B379F2187159F10126502906B225
:1004D000012703FB21F9237F06B371F2002650297F
:1004E0003150D0F006B2102713FB22F9277E16B345
:1004F00051F201265029012703FB06B223F92F7C74
:1005000049F2000006B3102713FB24F900265029F6
:1005100006B22F7939F270CF10E21ABF002717C048
:100520003B503195C31BD04010E21ABF0881033CF9
:10053000F9F00B34E9F0209186001981110F1213A4
:10054000EDCF093651F10D3211F0013E39F700932C
:100550008D003F915F914F911F910F912F91DF91EE
:100560000F90CAB7C5FD1DCFCF91CFBFCF911895C2
:1005700020918D00222369F310918B00112321F526
:10058000343022F130938B00209387001091880043
:100590003BE0311B3093880019C000918B00013083
:1005A0009CF40AE53091610034FD11C000936100B4
:1005B000CBE7D0E010C0052710E000C021C0052720
:1005C00010E0C89508BB14C03AE501C032ED032E17
:1005D000C0E0D0E032E017B31861C39A08B317BB8C
:1005E00058E120E84FEF20FF052708BB2795179516
:1005F0001C3F28F700004552B0F720FF052727953C
:1006000008BB17951C3FB8F629913A9561F7077E0C
:1006100010918C00110F08BBC250D04011F0109304
:10062000860010E21ABF086017B3177E402F477E7E
:1006300054E05A95F1F708BB17BB48BB8ACF582F37
:1006400048E080E057FD18C0C098550F880FB19959
:100650008F5FC29A32B72091AA0092B7931B92176C
:10066000E0F3C29832B72091AA0092B7931B921779
:10067000E0F3415039F70895C09AE7CFDC01CB0190
:1006800021E1B695A795979587952A95D1F7209161
:10069000A9002817D9F08093A900E091A600F09155
:1006A000A7008DE40995E091A600F091A70080E0F5
:1006B0000995E091A600F091A7008091A900099505
:1006C000E091A600F091A70080E0099408950895B4
:1006D0009FEF980F973050F08FE193E09093A70031
:1006E0008093A60082E08093AA0008952FE133E072
:1006F0003093A7002093A6008430F1F048F08630B4
:10070000C1F090F08730A1F483E08093AA000895AF
:10071000823031F0833061F480E38093AA00089541
:1007200080E68093AA0008958CE08093AA00089543
:1007300080EC8093AA00089588E18093AA00089530
:1007400022B79091AA0082B7821B8917E0F308951F
:10075000BD9ABA9AB89AC598C29822B79091AA0041
:1007600082B7821B8917E0F3C59A22B79091AA003D
:1007700082B7821B8917E0F3C5981092A9000895EB
:10078000BD98BA98B898C598C298C0980895CF9364
:10079000DF93C0E2E091A600F091A7008CEA0995F2
:1007A000E091A600F091A70083E50995E091A600ED
:1007B000F091A70080E00995D82FE091A600F09174
:1007C000A70080E00995D335E9F022B79091AA00FF
:1007D00082B7821B8917E0F3C59A22B79091AA00CD
:1007E00082B7821B8917E0F3C59822B79091AA00BF
:1007F00082B7821B8917E0F3C15061F681E0DF9177
:10080000CF91089580E0DF91CF910895CF92DF924C
:10081000EF92FF926B017C0131DF8C2D8170880F8C
:10082000880F880FE091A600F091A70080620995DB
:10083000D701C60129E0B695A795979587952A9582
:10084000D1F7E091A600F091A7000995D701C60164
:10085000B695A79597958795E091A600F091A7008A
:100860000995E091A600F091A70080E0FF90EF903D
:10087000DF90CF900994CF92DF92EF92FF920F9387
:100880001F93CF93DF931F92CDB7DEB76B017C012F
:10089000142F2983F3DE9C2D9170892F880F880FE8
:1008A000880FE091A600F091A70080640995D70118
:1008B000C60129E0B695A795979587952A95D1F712
:1008C000E091A600F091A7000995D701C601B69561
:1008D000A79597958795E091A600F091A7000995B7
:1008E000E091A600F091A700812F0995298122238C
:1008F000A9F01F3789F002B71EE1C701B60186DFF4
:100900008F3761F482B7801B843510F002B7115025
:100910001111F3CF81E003C08FE0B3D080E00F90DE
:10092000DF91CF911F910F91FF90EF90DF90CF90CB
:100930000895CF92DF92EF92FF920F931F93CF9380
:10094000DF931F92CDB7DEB76B017C01498396DE42
:10095000E091A600F091A7008CE40995D701C601AB
:1009600029E0B695A795979587952A95D1F7E091B7
:10097000A600F091A7000995D701C601B695A795E5
:1009800097958795E091A600F091A7000995E091D1
:10099000A600F091A70080E0099549814F3FE1F062
:1009A00002B71EE1C701B60131DF8F3F99F482B76C
:1009B000801B843510F002B711501111F3CF81E084
:1009C0000F90DF91CF911F910F91FF90EF90DF90EB
:1009D000CF90089580E0F4CF8FE053D080E0F0CF47
:1009E0001F93CF93DF931F92CDB7DEB7182FE091FF
:1009F000A600F091A70080EA99830995E091A600EE
:100A0000F091A7009981892F0995E091A600F091B6
:100A1000A700812F0995E091A600F091A70080E042
:100A20000F90DF91CF911F9109941F93CF93DF9384
:100A300000D0CDB7DEB7182FE091A600F091A70047
:100A400080EC6A8399830995E091A600F091A70054
:100A50009981892F0995E091A600F091A700812F37
:100A60000995E091A600F091A7006A81862F09956B
:100A70008EE107D080E00F900F90DF91CF911F9112
:100A80000895882349F030E022B792B7921B93353E
:100A9000E0F33F5F3813F8CF0895BA9AB898C09A38
:100AA00050E217D05A95E9F70895AC0188E605D0D1
:100AB000842F03D089E601D0852F0FD028E030E0C5
:100AC000382780FB869506D02A95D1F730FB02D0D7
:100AD00000D06894B898C09A16F0C098B89AE0917F
:100AE000AC00F091AD003197F0F7C29AE6B3E0FBAD
:100AF000E091AC00F091AD003197F0F7C298089505
:100B000020ECE7DF46F42A95E1F780E02AE1E5DF13
:100B10002A95E9F7DECF28E030E0DBDF869587F91C
:100B200038272A95D1F7D5DF27F9322772F3D1DF9D
:100B3000D0CFDB01742FB9DF84E2BFDFE1DF8D931B
:100B40007A95D1F70895DB01742FAFDF83EFB5DF1E
:100B50008DE1B3DF84E6B1DF8D91AFDF82E7ADDFFA
:100B6000CFDF8078D9F77A9589F70895CF93DF930F
:100B7000EC0199818FEB890F8430B8F19A35A9F196
:100B8000913009F4EEC0923009F4F3C0933009F4C7
:100B900074C0943009F4B8C0973009F490C095300F
:100BA00009F481C1963009F434C1983009F4F9C0D0
:100BB000993009F482C19A3009F4B1C19B3009F42B
:100BC000ECC19C3009F40DC29D3009F425C29E3061
:100BD00009F427C29F3009F481C1903109F4A6C1FC
:100BE0009F3709F4CFC180E014C020916200211129
:100BF00019C06A816A3F39F18823E1F1923409F022
:100C0000A8C06093B9008091B6008F5F8093B60052
:100C100084E023E730E030938A0020938900DF915D
:100C2000CF910895109262001FBC83E68DBD8BE8C2
:100C300080BF82E887B987E886B999818FEB890FF1
:100C40006A816A3FC9F6811197C086B3827080932A
:100C500073009091AF00909375009091BE009093B7
:100C60007600882319F081E080937300109274005D
:100C700084E0CFCF6093B800C6CFE091A600F0919A
:100C8000A7008A81099580937300E091A600F091F6
:100C9000A7008B81099580937400E091A600F091E4
:100CA000A7008C81099580937500E091A600F091D2
:100CB000A7008D8109958093760084E0AACF80916A
:100CC0007000811112C08B8190E0982F88272A81B3
:100CD000822B092E000CAA0BBB0B80936C00909307
:100CE0006D00A0936E00B0936F008F8190E0982FFD
:100CF00088272E81822B90936B0080936A0083E07B
:100D0000809372008FEF85CF80917000811112C0A7
:100D10008B8190E0982F88272A81822B092E000C46
:100D2000AA0BBB0B80936C0090936D00A0936E0098
:100D3000B0936F008F8190E0982F88272E81822BAF
:100D400090936B0080936A0082E0809372008FEF33
:100D500060CF933419F1943409F0AAC06093B700BE
:100D600052CF80917100B4DC10927000F1DC80E011
:100D700050CF06DD80E04DCF9234F1F1933409F08D
:100D800085C086B38072809373009091B300909376
:100D900075009091C2009093760063CF6093BC0081
:100DA00032CF80917000811112C08B8190E0982F1A
:100DB00088272A81822B092E000CAA0BBB0B80935B
:100DC0006C0090936D00A0936E00B0936F00109232
:100DD000690010926800109267008F8190E0982F50
:100DE00088272E81822B90936B0080936A0084E089
:100DF000809372008FEF0DCF86B384708093730061
:100E00009091B000909375009091BF009093760000
:100E100028CF80917000811112C08B8190E0982FB3
:100E200088272A81822B092E000CAA0BBB0B8093EA
:100E30006C0090936D00A0936E00B0936F003C81A6
:100E40002D81822F8F7080936700822F807F90E0AA
:100E500082959295907F9827807F9827830F911D88
:100E6000909369008093680020FD809366008F81D5
:100E700090E0982F88272E81822B90936B0080938F
:100E80006A0081E0809372008FEFC3CE943409F43E
:100E90006EC08FE090E085D38093750080937300DF
:100EA00010927600DECE73DC8093730081E0B1CEC9
:100EB0008FE090E07ED384E0ACCE81E08093700040
:100EC0008A819B81AC81BD8180936C0090936D0081
:100ED000A0936E00B0936F0080E09BCE8B8190E07A
:100EE000982F88272A81822B092E000CAA0BBB0B76
:100EF00080936C0090936D00A0936E00B0936F0090
:100F00008F8190E0982F88272E81822B90936B0001
:100F100080936A0085E0809372008FEF7ACE8A8199
:100F2000809371001092730081E073CE8B8190E00A
:100F3000982F88272A81822B092E000CAA0BBB0B25
:100F400080936C0090936D00A0936E00B0936F003F
:100F50008F8190E0982F88272E81822B90936B00B1
:100F600080936A0086E0809372008FEF52CE86B342
:100F7000817080937300811148C0109275001092A7
:100F8000760074CE81E0809373001092740010920A
:100F900075001092760084E03CCE8B8190E0982F13
:100FA00088272A81822BAC015695479556954795FF
:100FB0009C01369527953695279536952795240FCC
:100FC000351F820F931F9093AD008093AC00C59A9C
:100FD000BD9A83E056DDC59880E153DD5EDD80E09B
:100FE00018CE80EC6ADD80E068DD8AE04ADDC59AD3
:100FF00085E047DDC59885E044DDBD98BA98B8988E
:10100000C598C298C09880E004CE8FEF8093750099
:1010100083E08093760027CE73DD8093730081E0B8
:10102000F8CD8A814ADD80E0F4CDFF920F931F93C3
:10103000CF93DF93582F792FF62E209172003EEF39
:10104000320F323050F0253009F452C08FEFDF916B
:10105000CF911F910F91FF900895662309F43FC02F
:1010600080916C0090916D00A0916E00B0916F0026
:10107000052F172F3FEF360FE801C30FD11D1DC0FD
:10108000AFDCF801808380916C0090916D00A0919D
:101090006E00B0916F000196A11DB11D80936C0090
:1010A00090936D00A0936E00B0936F000C171D0716
:1010B00061F0209172000F5F1F4F223009F7BC01D1
:1010C000CD01A4DBF8018083DECFF7E0FF1538F413
:1010D0008F2DDF91CF911F910F91FF900895109266
:1010E00072008F2DDF91CF911F910F91FF90089586
:1010F000462F682F80916C0090916D001ADD8091D1
:101100006C0090916D00A0916E00B0916F008F0DFA
:10111000911DA11DB11D80936C0090936D00A09353
:101120006E00B0936F008F2D92CFFF920F931F939D
:10113000CF93DF93382F792F162F20917200213013
:1011400061F0243051F0263009F494C08FEFDF9124
:10115000CF911F910F91FF900895112309F482C040
:1011600080916C0090916D00A0916E00B0916F0025
:10117000C32FD72F1150AE01410F511D8A01F12C01
:101180004DC02091680030916900232B09F04FC0B9
:1011900021E04881BC01CD016EDB20916A003091D5
:1011A0006B002150310930936B0020936A00232B90
:1011B000E1F4109272008091670081FF35C0809148
:1011C000660090E0209168003091690082179307D3
:1011D00059F160916C0070916D0080916E0090915A
:1011E0006F004881A6DBFF24F39480916C009091FE
:1011F0006D00A0916E00B0916F000196A11DB11D10
:1012000080936C0090936D00A0936E00B0936F007C
:10121000C017D10741F1209172002196213009F4C5
:10122000B0CF688102DCB9CFFF24F394DECF20E099
:101230004881BC01CD011FDB809166008150809305
:1012400066008111AACF60916C0070916D00809151
:101250006E0090916F0048816CDB809168008093F4
:1012600066009BCFF12C8F2DDF91CF911F910F91B5
:10127000FF900895462F682F80916C0090916D002B
:1012800062DC80916C0090916D00A0916E00B09135
:101290006F00810F911DA11DB11D80936C00909373
:1012A0006D00A0936E00B0936F0080916A009091E2
:1012B0006B00811B910990936B0080936A00892BCE
:1012C00021F41092720081E042CF80E040CFEF9293
:1012D000FF920F931F93CF93DF9381B7D0E0C0E0CD
:1012E00080E1F82E0AC08D2F8160D1FDF694CF0DDC
:1012F000D82FC1BF81E08F15A0F43DD88C010433F5
:1013000089E0180784F3043399E0190751F08D2F11
:101310008260D0FDF694CF19D82FC1BF81E08F1520
:1013200060F38FEF8C0F81BF81B7EC2EF12C9FEF14
:10133000E91AF90A90E0E816F90674F416C0801765
:10134000910714F4C1B78C0181B78F5F81BF81B75A
:1013500090E0E816F9064CF00ED88453994097FFB8
:10136000EECF919581959109EACFC1BFDF91CF91E1
:101370001F910F91FF90EF90089583E083BF18BAFB
:1013800017BA8FEF87BB84E67CDB17BAC6D78EEF20
:101390008093B8001092AF001092BE008093B90005
:1013A0001092B0001092BF008093BC001092B30066
:1013B0001092C2008093B7001092AE001092BD0050
:1013C0001092B6001092B5001092B400789410E814
:1013D000D3E8C2E869D69FB58091B400981709F4A4
:1013E00056C08F5F843609F4AAC08093B400809100
:1013F000B8009FEF980F933658F42091B40030E076
:10140000082E000C990B281739070CF0BAC0C19AA6
:101410008091B9009FEF980F933658F42091B40053
:1014200030E0082E000C990B281739070CF0AFC0DC
:10143000C29A8091BC009FEF980F933658F4209188
:10144000B40030E0082E000C990B281739070CF077
:101450009AC0C59A8091B7009FEF980F933658F4C1
:101460002091B40030E0082E000C990B28173907A2
:101470000CF08BC0C09A18D68091B400833009F468
:1014800075C0843209F467C0853409F45BC00CD69A
:101490008091B5009091B600981709F49BCF8F5FAB
:1014A0008093B5008091B80087FD44C0811128C0A9
:1014B000C198B99A8091B90087FD26C081111CC0DE
:1014C000C298BA9A8091BC0087FD27C0811110C0D4
:1014D000C598BD9A8091B70087FD27C0811103C0D0
:1014E000C098B89A77CF8436E1F7C09AB89A72CF8D
:1014F000843679F7C59AEDCF843619F7C29AE1CFD1
:101500008436B9F6C19AD5CFBA988F3F09F441C055
:10151000C29A8091BC0087FFD9CFBD988F3FD9F187
:10152000C59A8091B70087FFD9CFB8988F3FB9F19E
:10153000C09A50CFB9988F3F81F1C19ABBCF10921A
:10154000B40055CF84B18093B00085B18093BF00C3
:1015500017B9369A9CCF84B18093AF0085B1809340
:10156000BE00D7B9369A8091B4008ECF84B18093F3
:10157000B30085B18093C200C7B9369A8091B40098
:1015800080CFC19845CFC59865CFC09874CFC29819
:1015900050CFC29897CFC5989DCFC1988BCFC09898
:1015A00019CFE199FECF9FBB8EBBE09A99278DB3EF
:1015B0000895262FE199FECF9FBB8EBBE09A01973D
:1015C0000DB2021639F01CBA2DBB0FB6F894E29A90
:0A15D000E19A0FBE0895F894FFCFD2
:0415DA00FF5A0100B3
:00000001FF
